:020000040000FA
:02000000BA281C
:08000800D129B30000308A0089
:10001000330882074E347234583469346134D13431
:100020006A34B234733413347A34FB348234733424
:1000300089347F349034263496346C349C345A346A
:10004000A134F134A7343934AC343434B034E83426
:10005000B5345934B9348934BD347E34C1343A347A
:10006000C434C034C8341334CB343634CE342D3495
:10007000D034F934D3349D34D6341A34D83474346B
:10008000DA34AD34DC34C534DE34BF34E0349D348E
:10009000E2346034E4340A34E5349B34E734173412
:1000A000E8347D34E934CE34EB340D34EC343A3476
:1000B000ED345734EE346334EF346034F0344F347D
:1000C000F1343034F2340534F234CE34F3348B343A
:1000D000F4343E34F434E734F5348734F6341D34E4
:1000E000F634AB34F7343134F734B034F8342734E1
:1000F000F8349834F9340334F9346734F934C634B5
:10010000FA341F34FA347434FA34C434FB340F3400
:10011000FB345634FB349934FB34D834FC34143477
:10012000FC344C34FC348134FC34B434FC34E334DB
:10013000FD341034FD343A34FD346234FD348834F7
:10014000FD34AB34FD34CD34FD34EC34FE340A34AC
:10015000FE342634FE344134FE345A34FE347234D4
:10016000FE348834FE349D34FE34B134FE34C4345D
:10017000FE34D63403138312850107309F008316A3
:100180001C308500FF308600403081000C10831247
:1001900001309000850186018B120B178B17851992
:1001A000CF280608FF3AF039A000A00E0608FF3A53
:1001B0000F39A1000310200DA107A00DA00D200DE7
:1001C000A10762302102031DE928FD2000308A00CA
:1001D000CF2863302102031DF1281F2100308A003F
:1001E000CF280C3021020318F928402100308A0062
:1001F000CF282D2100308A00CF28AE2183160C1481
:1002000083120130A4002408A600A6030310260DC3
:100210000520A2000314260D0520A3003230AC00F7
:10022000C421AC0B1029851D1A29A40A2408583CA6
:100230000318032983160C108312AE210800A001B5
:100240002008A100402185192729AE212C29A00AC8
:100250000C302002031C202908006130A10001306D
:10026000AF003530B00040210800C0341434C13430
:100270000334203404342734043480340434003408
:10028000AE210130A7006130210203195729031064
:10029000A10D0130AD00E1302107AE000318AD0A19
:1002A0009721AF00AE0A0319AD0A9721B000A12132
:1002B000A400240803198D29A121A500803024025F
:1002C00003198029C0302402031D69292508A600CE
:1002D0008A29C1302402031D74292F08B100300877
:1002E000B2002508A7008A29A4030310240D0520C5
:1002F000A2000314240D0520A30083160C148312FE
:100300002608AC00BD21AC0B8229A50B80298316E1
:100310000C108312851957299529A70B9029952927
:100320003108AF003208B0005729AE2108009D21E6
:10033000B30001308A00330808002D088A002E0817
:100340008200AA21B30001308A003308B00A0319E1
:10035000AF0A08002F088A00300882000530AC0080
:100360000514CB210510CB21AC0BB0290800C630F9
:10037000A800BA29A80BB92908000530A900B7219F
:10038000C129A90BBF2908003230AA00B721C8290A
:10039000AA0BC62908000530AB00C421AB0BCD2940
:1003A0000800F000030EF100830122088F002308EB
:1003B0008E00023085060C10710E8300F00E700E58
:1003C00009000134F934023476340234C33403347E
:1003D000383403348B34043436340434B9340534BB
:1003E00034340534D1340634923407340D340734B0
:1003F0009E34C034463420340834803401342034F0
:100400000834253408342734083428340834273491
:100410000834253410342134083480340134213434
:100420000834203408341E34083420341034803426
:100430001034203408348034013420340834253416
:100440000834273408342834083427340834253451
:100450001034213408341E34083420340C348034F1
:1004600001342034043419341034803410341C34F2
:100470000834803401341C3408341B3408341934F3
:10048000083421340C3480340134213404342034D1
:1004900010341E3408342034083421340C348034B1
:1004A00001342134043420341034803410342034A6
:1004B0000834803401342034083425340834273497
:1004C00008342834083427340834253410342134CF
:1004D00008341E34083420340C3480340134203481
:1004E000043419341034803410340034C0342D34C2
:1004F000C13402341C3408342134083480340134CB
:10050000213418342334083425340834283408348A
:100510002D3408342A340834283410342A3408346A
:10052000213408348034013421341034233410341D
:100530002534203480341034253408342A340834E7
:10054000283418342A3408342D3408342A34083432
:10055000283408342A34083428340834253408343C
:100560002834083425340834213408342534083438
:1005700023340834213408348034013421342034C5
:10058000803410340034C03428342534103480349E
:100590000134253410342734203425341034803489
:1005A00001342534103427342034253410342734D2
:1005B00010342834103427341034253410342734C0
:1005C00008342534083421342034203410341C34C9
:1005D000103420341034213410342034103480345A
:1005E0000134203408341C3408341B3420342534BE
:1005F0001034273410342834103427341034253480
:10060000103427340834253408342134203420347D
:1006100010341C341034203410342134103420347D
:10062000103480340134203408341C3408341B3432
:1006300020342534103480340134253410342734E8
:1006400020342534103480340134253410342734D8
:1006500020348034103420341034213420342734B2
:100660000834253408342134103420342034003444
:10067000C03432341E3410341C3410341E34103460
:100680002034103423341034203410341E342034F9
:1006900020341034233410342534103423340834F7
:1006A000253408342A3410342734103425341034D7
:1006B00023341034203410342334103425342034BF
:1006C0002A341034283410342A342034203410349E
:1006D00023341034253410342334103420341834A7
:1006E000233408341E342034253410342834103494
:1006F0002A342034283410342A3410342534103469
:10070000233410342534103423340834203408348E
:100710001E3420340034C0342834203418342134BA
:10072000083425341034803401342534083421341D
:1007300008342034103421340834203408341E3472
:1007400010342034103425341034803401342534EE
:10075000083426340834253408342334083420344B
:1007600008342334083425343034803410342334AE
:1007700010348034013423341034253410342334BD
:10078000083425340834263420342A3410342634EE
:1007900008342A34083425341034803401342534A4
:1007A00008342634083425340834233408342034FB
:1007B0000834233408342534303480341034203461
:1007C0001034803401342034083421340834253482
:1007D0001034803401342534083421340834203472
:1007E000103421340834203408341E3410341934C1
:1007F00010342034103421340834203408341E34AA
:100800001034203408342134083425341834213489
:100810000834203410341E341034263418342A346A
:10082000083426341034253410342C3410342D344C
:1008300008342C3408342A341034263408342A344A
:1008400008342534103480340134253408342634F7
:10085000083425340834233408342034083423344D
:10086000083425343034803410340034C0341A3421
:1008700023341034203408341E3408342034103427
:1008800023340834253408342734203425341034F4
:100890008034103423341034803401342334083449
:1008A000253408342A3410342734103425340834DD
:1008B00023340834203408341E34083420341034EF
:1008C000803410341B341034803401341B34083429
:1008D000803401341B3408341E3408342034083486
:1008E000233408342034083425342034233410349D
:1008F000803410342534103423340834253408343B
:100900002734103423341034253408342334083485
:1009100020341034803401342034103480341034C6
:100920001E34103420340834233408342534103471
:100930002A341034273420342534103480341034D1
:1009400023341034803401342334083425340834FB
:100950002A3410342734103425340834233408342E
:10096000203408341E3408342034103480341034D9
:100970000034C0342234C1340234203408342334E7
:100980000834803401342334103480340134233467
:1009900020342034083423340834803401342334A0
:1009A0001034803401342334203480340834253426
:1009B0000834233408348034013423340834253493
:1009C0001034233408348034013423340834203480
:1009D00008342334083425340834213408342334CB
:1009E00020348034083420340834233408348034EC
:1009F0000134233408342034083423340834803458
:100A00000134233408348034013423340834253449
:100A10000834803401342534043427340434283431
:100A200008342A34083423342034803408342834F9
:100A3000083423340834203408341E340834253470
:100A400008348034013425340834803401342534AA
:100A500008342834083423340434203404341E3455
:100A60001034203420340034C0342D342034083481
:100A70008034013420340834803401342034083484
:100A800080340134203408342334043421340434D1
:100A90008034013421340434203404341E341034BE
:100AA000803401341E340834803401341E34083458
:100AB00020340834213408342334103428340834E2
:100AC000803408342034083480340134203408342D
:100AD0008034013420340834803401342034083424
:100AE0002334043422340434803401342234043472
:100AF000203404341E341034803401342334083458
:100B0000803401342334083425340C342334043441
:100B10002234043423340434253404342734043494
:100B2000233410348034013423340434273404341F
:100B3000253404342334043422340434203404347B
:100B40001F3404342034043428340C342234043464
:100B500023341034803401341E340834803401349A
:100B60001E34083420340834213408342334083443
:100B700025340434273404342834103480340134C8
:100B80002534083428340834213408342534083412
:100B90001C340834203404341E3404341C3410341F
:100BA0000034C03428341E34083423340834273445
:100BB000103480340134273408348034013427342D
:100BC0000834803401342734103425340834273471
:100BD00008342534083423341834803410341E3457
:100BE00008342334083427341034233408342734A9
:100BF00008342A341034283408342734083425348F
:100C000030342A34083428340834273410348034FB
:100C1000013427340834253408342334103425347F
:100C20000834273408342A340834283418348034FB
:100C30001034203408341F3408341E341034223465
:100C40000834233408342534103427340834253448
:100C500008342334303423340834803401342334CA
:100C60000834203410348034013420340834803483
:100C700001342034083480340134203410342334D7
:100C8000083480340134233408348034013423346C
:100C9000083480340134233418348034103423343D
:100CA000083480340134233408342234103480343E
:100CB000013422340834803401342234083420349E
:100CC00010342534083423340834223430342A34A0
:100CD000083428340834273410348034013427345D
:100CE00008342534083423341034253408342734A8
:100CF00008342A340834283418348034103420342A
:100D000008341F3408341E34103422340834233499
:100D10000834253410342734083425340834233477
:100D200030340034C0341C342334103427341034AD
:100D300022341034803401342234103420341034FE
:100D400022340834203408341B3410341B3410345B
:100D500023341034273410342234103480340134D6
:100D600022341034203410341F3410342034203412
:100D7000803420348034103423340834253408344B
:100D8000273410348034013427341034803408344C
:100D900028340834253408342334083422341834F1
:100DA0008034083423340834273410348034013438
:100DB0002734083480340134273408348034013433
:100DC00027340834253408342334083427342034B5
:100DD0002334103427341034223410348034013456
:100DE00022341034203410342234083420340834AF
:100DF0001B3410341B341034233410342734103493
:100E0000223410348034013422341034203410342D
:100E10001F341034203420340034C03423342334BD
:100E20001034203408342334083428342034253452
:100E300010342834083480340134283408342334FE
:100E4000203480340134233410341C3408341E34EC
:100E50000834203410341E3408341C3408341E3452
:100E600030348034103423341034203408342334A4
:100E700008342834183427340834253410342834FE
:100E800010342334203480340134233410341E349D
:100E9000083420340834213418341B3408341C340A
:100EA00030348034103425341034283408348034FD
:100EB0000134283408348034013428342034273471
:100EC00010342534083427340834283420342534A9
:100ED000083427340834283408342534083480345E
:100EE00001342534083423340834203408341C34C5
:100EF00008341E3430348034103423341034203419
:100F000008341C3408342834183427340834253481
:100F10001034283410342334203480340134233402
:100F200010341E34083420340834213418341B346F
:100F300008341C343034803410340034C034263447
:100F4000C1340234213418341F3408341E340834B8
:100F50002134083426340834283408342A34203420
:100F60002634203428340834263408342534083410
:100F700028340834263410342334103421343034E7
:100F800080341034213418341F3408341E340834AB
:100F900021340834263408342A34083428342034E0
:100FA00023342034253418342334083421340834CD
:100FB00025340834263408342834083426343034B0
:060FC000803410340034FF
:02400E00223F4F
:00000001FF
